:20010000C0A875A800850882850983F0A3E5F0F0A3E50AF0A3E50BF0A38582088583098595
:20012000820A85830BD0A822D0E0D0E0C0A875A800E50824FCF508E50934FFF509D0028521
:200140000882850983E0C0E0A3E0C0E0A3E0F50AA3E0F50BA38502A822C0A875A800C0D053
:2001600075D000C082C083C0E0C0F0C000C001850882850983E58124F5F8E6F0A308E6F0F6
:20018000A308E50AF0A3E50BF0A3080808E6F0A308E6F0A308E6F0A308E6F0A308E6F0A31A
:2001A00008E6F0A308E6F0A37900E7F0A309B90DF985820885830985820A85830BE58124B4
:2001C000F9F581D000D0F0D0E0D001D001C0E0C0F08500A82275D00085A80075A800E508B3
:2001E00024E8F508E50934FFF509850882850983D0E0D0E0E0C0E0A3E0C0E0A3C000E0F57C
:200200000AA3E0F50BA3E0C0E0A3E0C0E0A3E0C0E0A3E0C0E0A3E0C0E0A3E0C0E0A3E0C03C
:20022000E0A37900E0F7A309B90DF9D001D000D0F0D0E0D083D082D0D0D0A832D083D082DB
:20024000C082C083A3A3A3E5F070012215F0E493A365016006A3A3A3A380ECE493A3650066
:200260006005A3A3A380E0D0E0D0E0E473E501750100450070047500012275000022E501EF
:200280007501006503700AE500650270047500012275000022E501650330E727750100E530
:2002A0000320E7047500012275000022E501650330E726750100E50320E704750001227500
:2002C000000022C3E5009502E501950375010050047500012275000022C3E5029500E5031F
:2002E000950175010040047500012275000022E5002502F500E5013503F5012285028285BA
:200300000383E02401F0A3E03400F0222500F500E5013400F50122F5F0E500C395F0F50046
:20032000E5019400F50122E502540F6013F506C3E50033F500E50133F5011506E50670EF2F
:2003400022E502540F6013F506C3E50113F501E50013F5001506E50670EF22E5016503301F
:20036000E73012036C12039212036C22E501F4C0E0E500F42401F500D0E03400F50122E54D
:2003800003F4C0E0E502F42401F502D0E03400F50322E5018502F0A4C0E0E5008503F0A42F
:2003A000C0E0E5008502F0A4F500D0E025F0D0F025F0F50122750701E501450320E704122E
:2003C000044722E501550320E73BE50130E71B12036C12044712036CE50130E727E500258B
:2003E00002F500E5013503F5012212037F12044712036CE50130E70CE5002502F500E5016E
:200400003503F5012212036C12037F12044722750700E501450320E70412044722E5015589
:200420000320E719E50130E70A12036C12044712036C2212037F12044712036C2212036CFC
:2004400012037F12044722E5024503700122E50345017010E5008502F084F500E5076003F5
:2004600085F000227E01E503C320E70D0EE50233F502E50333F50380F0750400750500C052
:2004800000C001C3E5009502F500E5019503F501B3501DD0E0D0E0E50433F504E50533F54C
:2004A00005C3E50313F503E50213F502DED1801BD001D000E50433F504E50533F505C3E5D1
:2004C0000313F503E50213F502DEB4E507700685040085050122C0A875A8008508828509D1
:2004E00083E500F0A3E501F0A3858208858309D0A822C0A875A800850882850983E502F052
:20050000A3E503F0A3858208858309D0A822C0A875A800E50824FEF508F582E50934FFF5E5
:2005200009F583E0F502A3E0F503D0A822C0A875A8002508F508E50935F0F509D0A82225CF
:200540000AF582E50B35F0F583E0F500A3E0F50122250AF582E50B35F0F583E0F502A3E090
:20056000F503222502F582E50335F0F583E0F500A3E0F50122850282850383E500F0A3E55D
:2005800001F022E50CF50075010022C0A875A800850882850983C5F0F0A3E5F0F0A385826E
:2005A00008858309D0A822E500C0E0E501C0E0E502F500E503F501D0E0F503D0E0F5022252
:0105C0002218
:030000000205E115
:2005E10075811F020620D0F0D0E0120100750100E4A29092E0F500E500450170030206049D
:200601000205EE750100E4A29092E0F50012026DE5004501700302061D02060412012875F1
:20062100094075080085090B85080A740275F00012052D850A02850B037500007501001283
:200641000575750001750100740075F00012053F75020A750300120295E5004501700302C2
:200661000682750C001205E7740075F00012053F740112030C850A02850B031205750206F5
:2006810049D291740075F00012053F750214750300120295E500450170030206BD750C00EE
:2006A1001205E7740075F00012053F740112030C850A02850B03120575020684C291850A58
:1B06C10002850B0375000075010012057502064374FE75F0FF12052D02062085
:00000001FF
